:100000007328640017200318012822209401083067
:100010008F00232017200318940A971E94018E0C3A
:100020008F0B0928971A8E1323200E080800260824
:10003000840024088417800484130005171B2406F9
:10004000FF3E0800231717081F39FF3E8D001608D2
:10005000F53E03188D0A231F522823138C0002300B
:1000600069205228890083160814831208086E2814
:1000700088008316081555308900AA308900881435
:100080008818402808116E288F018E00FF308E07D7
:10009000031C8F07031C6E2803308D00DF305220B5
:1000A00046288D01E83E8C008D09FC30031C5B283E
:1000B0008C07031858288C0764008D0F58280C18DB
:1000C00061288C1C652800006528080003108D0C31
:1000D0008C0CFF3E031866280C086E28831303134C
:1000E0008312640008006400851CB5286400851C28
:1000F0007A28762801308F00F43045206400851C72
:100100008328A9017A290515831605110530831264
:10011000A6000130A4005430960040309700012022
:100120003A3C031D8F2801202A3C031D8F28012003
:100130003D3C031D8F2801204A3C031D8F280120D0
:100140003D3C031D8F280120313C031D8F280120D9
:10015000653C031D8F280120A80001308900280874
:100160003820051183160511831201303220A800B2
:1001700085158316851183120530A6000130A40071
:1001800054309600403097000120413C031DC428A4
:100190000120643C031DC42801202B3C031DC428FE
:1001A00001202B3C031DC4280120543C031DC428FE
:1001B00001207E3C031DC4280120213C031DC428CE
:1001C0000120AD00AA0164002A082D02031C792930
:1001D0000530A6000130A40054309600403097004E
:1001E0000120AC0064002A082802031D772964005E
:1001F00080302C02031C03298030AC028617831642
:1002000086138312072986138316861383126400CC
:1002100040302C02031C13294030AC020617831611
:10022000061383121729061383160613831264001C
:1002300020302C02031C23292030AC0286168316A2
:10024000861283122729861283168612831264006F
:1002500010302C02031C33291030AC020616831612
:1002600006128312372906128316061283126400BF
:1002700008302C02031C43290830AC028615831673
:100280008611831247298611831686118312640012
:1002900004302C02031C53290430AC0206158316CB
:1002A0000611831257290611831606118312640062
:1002B00002302C02031C63290230AC028614831620
:1002C00086108312672986108316861083126400B5
:1002D00001302C02031C7229AC030614831606108D
:1002E000831276290610831606108312BC28AA0FE3
:1002F000E328BC286400851C7E297A29640029082B
:100300000C3C031D8429A90164002908003C031D3D
:10031000A9290610831606108312861083168610EC
:100320008312061183160611831286118316861115
:100330008312061283160612831286128316861201
:1003400083120613831606138312861383168613ED
:10035000831264002908013C031DB2290614831688
:100360000610831264002908023C031DBF290610F1
:100370008316061083128614831686108312640077
:100380002908033C031DCC2986108316861083128E
:10039000061583160611831264002908043C031D08
:1003A000D929061183160611831286158316861124
:1003B000831264002908053C031DE6298611831673
:1003C000861183120616831606128312640029080A
:1003D000063C031DF32906128316061283128616A5
:1003E00083168612831264002908073C031D002A25
:1003F000861283168612831206178316061383123B
:1004000064002908083C031D0D2A061383160613F1
:100410008312861783168613831264002908093C09
:10042000031D322A061483160610831286148316BF
:1004300086108312061583160611831286158316FD
:1004400086118312061683160612831286168316E9
:1004500086128312061783160613831286178316D5
:1004600086138312051583160511831285158316CD
:1004700085116400831229080A3C031D5F2A0610B7
:1004800083160610831286108316861083120611B7
:1004900083160611831286118316861183120612A3
:1004A000831606128312861283168612831206138F
:1004B0008316061383128613831686138312640031
:1004C00029080B3C031D842A061483160610831288
:1004D0008610831686108312061583160611831262
:1004E000861183168611831206168316061283124E
:1004F000861283168612831206178316061383123A
:1005000086138316861383120130AB0064001A3001
:100510002B020318942A0A3044206400851C922A76
:10052000A90A7A29AB0F862A0511831605118312B1
:100530008511831685116400831229080A3C031D66
:10054000C12A061483160610831286148316861099
:1005500083120615831606118312861583168611DB
:1005600083120616831606128312861683168612C7
:1005700083120617831606138312861783168613B3
:100580008312640029080B3C031DE62A061083161B
:1005900006108312861483168610831206118316A2
:1005A000061183128615831686118312061283168E
:1005B000061283128616831686128312061383167A
:1005C0000613831286178316861383120130AB003D
:1005D00064001A302B020318F62A0A304420640003
:1005E000851CF42AA90A7A29AB0FE82A7A29630024
:0205F000F72AE8
:02400E00F53F7C
:00000001FF
